S123A100FFB455BDA81AFFB457A60026037EA275BDA9E57FB44CCE0000FFB567FFB44DFE95
S123A120B5636F00FFB565FEB457BDAA2C27037EA272CE0001FFB5617FB5717FB5697FB5C9
S123A1406ABDAAB624037EA1A3BDA5F17DB55B2714FEB55BBDA6632506BDA28E7EA272FEF4
S123A160B55BBDA62C7DB55D271CFEB55DBDA6B6BDA6FF2406BDA27E7EA272BDA3C82406F4
S123A180BDA27E7EA272FEB567F6B5713AFFB567FCB567F3B569FDB567FEB56108FFB5614E
S123A1A07EA13881002706CEB197BDA78AFEB457BDA81AA600270A812D2706FFB4577EA12F
S123A1C027FEB455BDA81AFFB4577CB44CCE0000FFB567FFB44DFEB457BDAA2C27037EA279
S123A1E072CE0001FFB5617FB5717FB5697FB56ABDAAB624037EA249BDA5F17DB55D271C53
S123A200FEB55DBDA6B6BDA6FF2406BDA27E7EA272BDA3C82406BDA27E7EA2727DB571278B
S123A22003BDA9CA7DB44F2703BDA310FEB567F6B5713AFFB567FCB567F3B569FDB567FE02
S123A240B56108FFB5617EA1E781002706CEB197BDA78AFEB457BDA81AA600270A812D27DB
S123A26006FFB4577EA1D67DB44F2703BDA699BDA2DE7ED003CEB05BBDA78A7EA2727DB417
S123A280502653BDA2FDCEB1C0BDA78A20487DB4502643BDA2FDCEB1D2BDA78A20387DB4F2
S123A2A0502633BDA2FDCEB1E4BDA78A20287DB44C27237DB450261EBDA2FDCEB1F6BDA73B
S123A2C08A20137DB44C270E7DB4502609BDA2FDCEB20BBDA78AFEB44D08FFB44D39FEB494
S123A2E04D2713CEB16CBDA78ACEB44DBDA7CABDA795BDA79539CEB177BDA78A39FEB457AC
S123A300BDA778BDA7C2CEB561BDA7CABDA7C239CEB561BDA7CABDA7C2CEB567BDA7BE7F03
S123A320B43FBDA364BDA7C2BDA7C2CEB459BDA78ABDA795B6B571B1B43F2727BDA7C2BDA3
S123A340A7C2BDA7C2BDA7C2BDA7C2BDA7C2BDA7C2BDA7C2BDA7C2BDA7C2BDA7C2BDA38B4F
S123A360BDA795395FCEB572F1B571270DC1042719BDA7C05CF7B43F20EEC104270CBDA72F
S123A380C2BDA7C2BDA7C25C20F039F6B43FCEB5723AF1B571270ABDA7C05CC50327032014
S123A3A0F139BDA795BDA7C2BDA7C2BDA7C2BDA7C2BDA7C2BDA7C2BDA7C2BDA7C2BDA7C220
S123A3C0BDA7C2BDA7C220CA7FB571FEB56FA6092A037EA4F8810527458104274DFEB55F89
S123A3E0A600812326037EA457812C26037EA48DA601812C26037EA48DA602812C26037EC0
S123A400A48DA603812C26037EA48DFEB55FA600813C27037EA4B208FFB55F7EA4D4A608A7
S123A420B7B5728601B7B5710C39A604B7B5728602B7B571FEB55FBDA83924037EA5ECFCC2
S123A440B44AB3B567830002F7B5734D270781FF2703BDA2C30C39FEB56FA60426037EA4E4
S123A460F6B7B572A6094CB7B571FEB55F08BDA83924037EA5ECB6B57181022708FEB44AB4
S123A480FFB5730C39B6B44BB7B5730C39FEB56FA6062762B7B5728602B7B571FEB55FBD0A
S123A4A0A839B6B44BB7B5737DB44A2703BDA2AE0C39FEB56FA607273DB7B5728603B7B526
S123A4C071FEB55FBDA83924037EA5ECFEB44AFFB5730C39FEB56FA605271BB7B572860244
S123A4E0B7B571FEB55FBDA83924037EA5ECB6B44BB7B5730C390D39818026037EA52B817D
S123A5008426037EA53E818526037EA551818126037EA575818226037EA59B818326037E2E
S123A520A5C4818626037EA5EA0D39FEB55FBDA83924037EA5ECFEB44AFFB5670C39FEB536
S123A5405FBDA83924037EA5ECFCB44AFDB5690C39FEB55FBDA83924037EA5ECFEB55BBDB9
S123A560A66324037EA29EFEB443BDA81A08FCB44AED000C39FEB55FBDA83924037EA5EC5B
S123A580B6B44BCEB572F6B5713AA7007CB571FEB448A60008812C27DF0C39FEB55FBDA857
S123A5A03924037EA5ECCEB572F6B5713AFCB44AED007CB5717CB571FEB448A60008812C5D
S123A5C027DC0C39FEB55FA600B7B43F08A6002717B1B43F27123CCEB572F6B5713AA700D6
S123A5E07CB57138270220E40C390C39BDA2AE0C39CE0000FFB55BFFB55DFFB55FCEB45998
S123A600A6002727812A2723813B271F8120270781092703FFB55BBDA81A6D00270DFFB5E5
S123A6205DBDA81A6D002703FFB55F39A600BDA9B5251EA600271A8120271681092712814A
S123A6403A270E3CFEB565A70008FFB565380820E2FEB5656F00FCB567ED010808086F0015
S123A660FFB565FFB441FEB563FFB4436D002721BDA717240EFEB443BDA81A080808FFB41C
S123A6804320E9FEB443BDA81A08EE00FFB4450C397FB4457FB4460D39CEB160BDA78AFEC1
S123A6A0B5636D00270FBDA78A08BDA7C2BDA7BEBDA79520ED39A60084DFB7B56BA6018453
S123A6C0DFB7B56CA60284DFB7B56DA6038140230A817A220684DFB7B56E39862020F8A647
S123A6E000B1B56B2617A601B1B56C2610A602B1B56D2609A603B1B56E26020C390D39C6F9
S123A7000ACEAAEC6D00270DBDA6DF24033A20F4FFB56F0C390D39FEB4413CFEB4433CFE63
S123A720B443A6008D30271B3CFEB441E60008FFB441381126030820E938FFB44338FFB4CC
S123A740410D39FEB441A6008D0C26ED38FFB44338FFB4410C394D271D8120271981092767
S123A7601581202711813A270D812C2709812B2705812D2701394F39A600271881202714EB
S123A78081092710BD7FE80820EEA6002706BD7FE80820F63936860DBD7FE8860ABD7FE8CB
S123A7A0323944444444840F8B30813923028B277E7FE8A600BDA7A2A600087EA7A68DF3B1
S123A7C08DF1368620BD7FE832397FB4528604B7B453EC00CEA8128D0B08087AB45326F705
S123A7E0177EA7A67FB454A100250D2204E1012507A3007CB45420EF36B6B454260C7DB458
S123A8005226078630BD7FE820067CB452BDA7A63239271003E80064000AA60027178120A9
S123A8202707810927030820F1A60027088120270581092701390820F07FB44A7FB44B86F3
S123A8402BB7B447A600812B2606B7B447082008812D2604B7B44708FFB448A600812427B8
S123A860298125272F81272730812A2737BDA9B5251D7DB44C270ABDA6632403BDA29E2092
S123A8802C7FB44A7FB44B0C2023BDA8F7201EBDA9272019BDA96A201408A600B7B44B7FF7
S123A8A0B44A2038FCB567FDB4450C20002532B6B447812D2608FCB44AB3B4452006FCB4A4
S123A8C04AF3B445FDB44ABDA8E6A600270E812B26037EA83F812D26037EA83FFFB4480CA0
S123A8E039FFB4480D39FEB448A600BDA75627030820F6FFB448397FB4457FB446A60081EC
S123A90024260108A600BDA7562718BDA99B2415FDB43FFCB44505050505FAB43FFDB4452B
S123A9200820E10C390D397FB4457FB446A600BDA756271EBDA99B241B81092E17BDA9561E
S123A9407FB43FB7B440FCB445F3B43FFDB4450820DB0C390D393637FCB44505FDB43F051B
S123A96005F3B43FFDB4453332397FB4457FB446A6008125260108A600BDA7562719BDA9E2
S123A9809B24D181012E12B7B43FFCB44505FAB43FFDB4450820E00C390D39271680302B2F
S123A9A01281092F0C84DF81112D0881162E0480070D390C3936815F270A84DF8140230722
S123A9C0815A2E03320C39320D397DB45127155FF1B571270FCEB5723AA600FEB5673AA73E
S123A9E0005C20EC39CE0100FFB563FEB455A600272C812D2705BDA81A20F308A60084DF4F
S123AA00814C26037CB44F814526037CB450814426037CB45181542603BDAA1F20D8390822
S123AA20BDA8F725F9FCB445FDB56339FFB223FFB235CEB221BDD0067DB2222615B6B2254E
S123AA4085402618CE0000FFB23BFFB23DFFB2394F39CEB186BDA78AB6B22239CEB1A9BD3A
S123AA60A78A86FF39FEB23BBCB2282246FEB23DBCB22A273E188401188C00002612CEB217
S123AA8033BDD0067DB234262BFEB23908FFB239FCB23D8401C3B23F18A60018FCB23DC3B5
S123AAA00001FDB23D2409FCB23BC30001FDB23B180C394F0D39CEB459FFB559BDAA652516
S123AAC01F810A2714810D27F3FEB559A700088CB5582205FFB55920E3FEB5596F000C399A
S123AAE0FEB5598CB45926F16F000D39414444418B9BABBB000141444442CBDBEBFB0001B2
S123AB0041444444C3D3E3F3000241424120000000001B05414443418999A9B9000141449F
S123AB204342C9D9E9F90001414E44418494A4B40001414E4442C4D4E4F4000142495441DC
S123AB408595A5B5000142495442C5D5E5F50001434C522000006F7F0000434C52410000D5
S123AB6000004F05434C5242000000005F05434D50418191A1B10001434D5042C1D1E1F1EA
S123AB80000143424120000000001105434F4D20000063730000434F4D4100000000430577
S123ABA0434F4D420000000053054E4547200000607000004E4547410000000040054E455B
S123ABC04742000000005005444141200000000019054445432000006A7A000044454341B2
S123ABE0000000004A0544454342000000005A05454F52418898A8B80000454F5242C8D826
S123AC00E8F80000494E432000006C7C0000494E4341000000004C05494E434200000000E6
S123AC205C054C4441418696A6B600014C444142C6D6E6F600014C444420CCDCECFC000212
S123AC404D554C20000000003D054F5241418A9AAABA00014F524142CADAEAFA00015053A4
S123AC6048410000000036055053484200000000370550554C4100000000320550554C4207
S123AC80000000003305524F4C20000069790000524F4C41000000004905524F4C420000DE
S123ACA000005905524F5220000066760000524F5241000000004605524F5242000000008F
S123ACC0560541534C2000006878000041534C4100000000480541534C4200000000580548
S123ACE041534C440000000005054153522000006777000041535241000000004705415337
S123AD0052420000000057054C5352200000647400004C5352410000000044054C535242A8
S123AD200000000054054C535244000000000405535441410097A7B700005354414200D759
S123AD40E7F700005354442000DDEDFD0000535542418090A0B0000153554242C0D0E0F027
S123AD600001535542448393A3B3000253424120000000001005534243418292A2B20001A5
S123AD8053424342C2D2E2F200015441422000000000160554424120000000001705545360
S123ADA0542000006D7D000054535441000000004D0554535442000000005D0541494D200D
S123ADC00071610000034F494D2000716100000345494D2000756500000354494D20007B63
S123ADE06B000003435058208C9CACBC000244455820000000000905444553200000000039
S123AE003405494E5820000000000805494E53200000000031054C445820CEDEEEFE0002F7
S123AE204C4453208E9EAEBE00025354582000DFEFFF000053545320009FAFBF00005458B2
S123AE4053200000000035055453582000000000300541425820000000003A055053485870
S123AE60000000003C0550554C58000000003805584744580000000018054252412020009A
S123AE800000000442524E2021000000000442434320240000000004424353202500000056
S123AEA00004424C4F2025000000000442455120270000000004424745202C000000000423
S123AEC0424754202E000000000442484920220000000004424C45202F0000000004424C72
S123AEE05320230000000004424C54202D0000000004424D49202B0000000004424E452065
S123AF00260000000004425643202800000000044256532029000000000442504C202A007C
S123AF2000000004425352208D00000000044A4D502000006E7E00004A535220009DADBD68
S123AF4000004E4F502000000000010552544920000000003B055254532000000000390534
S123AF6053574920000000003F0557414920000000003E05534C5020000000001A05434C75
S123AF804320000000000C05434C4920000000000E05434C5620000000000A05534543201F
S123AFA0000000000D0553454920000000000F0553455620000000000B0554415020000043
S123AFC000000605545041200000000007054F5247200000000000804643422000000000DE
S123AFE000814644422000000000008246434320000000000083524D42200000000000846A
S123B00045515520000000000085454E4420000000000086535043200000000000864E4104
S123B0204D200000000000864E414D4500000000008654544C200000000000864F505420C5
S123B040000000000086504147200000000000865041474500000000008600363330312F4C
S123B0603633303320617373656D626C65722076312E302E320D0A44616E69656C20547550
S123B08066766573736F6E20323031372D323032320D0A53796E7461783A2061736D205B17
S123B0A066696C65735D205B2D6C5D205B2D655D205B2D645D205B2D74585858585D0D0AE8
S123B0C04F7074696F6E733A0D0A20202D6C2020202020205072696E74206C697374696ED6
S123B0E0670D0A20202D6520202020202048696465206572726F72730D0A20202D642020DD
S123B10020202020417373656D626C65206469726563746C7920746F206D656D6F72790D36
S123B1200A20202D745858585820204D6F76652073796D626F6C207461626C6520746F20E8
S123B14061646472657373202458585858202864656661756C74202430313030290D0A00EF
S123B1600D0A4C6162656C733A0D0A000D0A4572726F72733A20000D0A4E6F206572726F76
S123B18072730D0A0A0046696C65206E6F7420666F756E640D0A0046696C65207265616425
S123B1A0206572726F720D0A00456E7472792069732061206469726563746F72790D0A008F
S123B1C0496E76616C6964206F702D636F64650D0A004475706C6963617465206C61626577
S123B1E06C0D0A004C6162656C206E6F7420666F756E640D0A00496E76616C696420657860
S123B2007072657373696F6E0D0A004272616E6368206F7574206F662072616E67650D0AA1
S122B2200001000000000000000000000000000000000011000000B23F00000000000008
S116B43F00000000000000000000000000000000000000F6
S9030000FC
